:0200000480007A
:100000006F00C004732F2034930F8000630AFF0336
:10001000930F90006306FF03930FB0006302FF038A
:10002000170F0080130F0FFE63040F0067000F000F
:10003000732F203463540F006F004000136E9E53E3
:10004000171F00002320CFFD6FF09FFF732540F1A5
:100050006310050073251030635805000F00F00F82
:10006000130E100073000000130E00009702000032
:10007000938282F973905230735020307350303035
:1000800073504030970200809382C2F7638C020065
:10009000739052109302B01A739022307323203061
:1000A000E39E62F873500030970200009382420191
:1000B00073901234732540F17300203097200000B4
:1000C000938040F483A10000B70EFF00938EFE0FD3
:1000D000130E2000639AD12797200000938080F2AE
:1000E00083A14000B70E01FF938E0EF0130E300077
:1000F000639CD125972000009380C0F083A18000ED
:10010000B71EF00F938E0EFF130E4000639ED12397
:1001100097200000938000EF83A1C000B7FE0FF08E
:10012000938EFE00130E50006390D12397200000A1
:10013000938000EE83A140FFB70EFF00938EFE0F69
:10014000130E60006392D12197200000938040EC51
:1001500083A180FFB70E01FF938E0EF0130E700087
:100160006394D11F97200000938080EA83A1C0FF91
:10017000B71EF00F938E0EFF130E80006396D11DF5
:10018000972000009380C0E883A10000B7FE0FF025
:10019000938EFE00130E90006398D11B97200000F1
:1001A000938040E6938000FE83A10002B70EFF001B
:1001B000938EFE0F130EA0006398D11997200000B4
:1001C000938040E49380D0FF83A17000B70E01FFBD
:1001D000938E0EF0130EB0006398D117130EC0006B
:1001E0001302000097200000938000E283A14000EA
:1001F00013830100B71EF00F938E0EFF6316D31505
:100200001302120093022000E31E52FC130ED000D2
:100210001302000097200000938040DF83A140007C
:100220001300000013830100B7FE0FF0938EFE0051
:10023000631CD3111302120093022000E31C52FC32
:10024000130EE0001302000097200000938080DB73
:1002500083A140001300000013000000138301007D
:10026000B70E01FF938E0EF06310D30F130212002E
:1002700093022000E31A52FC130EF0001302000058
:1002800097200000938040D883A14000B71EF00F54
:10029000938E0EFF639AD10B13021200930220007B
:1002A000E31052FE130E000113020000972000001D
:1002B0009380C0D51300000083A14000B7FE0FF06B
:1002C000938EFE006392D109130212009302200064
:1002D000E31E52FC130E10011302000097200000D1
:1002E000938040D2130000001300000083A140005F
:1002F000B70E01FF938E0EF06398D1051302120022
:1003000093022000E31C52FC97210000938181CFCF
:1003100003A1010013012000930E2000130E200101
:100320006314D103972100009381C1CD03A1010083
:100330001300000013012000930E2000130E300163
:100340006314D101631CC0010F00F00F63000E00A5
:10035000131E1E00136E1E00730000000F00F00F2E
:10036000130E100073000000731000C000000000A6
:10037000000000000000000000000000000000007D
:040380000000000079
:1010000000000000000000000000000000000000E0
:1010100000000000000000000000000000000000D0
:1010200000000000000000000000000000000000C0
:1010300000000000000000000000000000000000B0
:081040000000000000000000A8
:10200000FF00FF0000FF00FFF00FF00F0FF00FF0D8
:040000058000200057
:00000001FF
